:020000040000FA
:02000000142AC0
:08000800A900030E8301AA0008
:100010000A08F0000408F1008312031386158C1EF1
:10002000012A181D14281628981C1B28181198102E
:1000300018121816012A1A08AC002C087F398207FA
:10004000012A012A012A012A012A012A012A012A58
:10005000012A012AA028012A012AA028012A012A0E
:10006000012A012A012A012A012A012A012A012A38
:10007000012A012A012A012A012A012A012A012A28
:10008000012A012A012A012A012A012A012A012A18
:10009000012A012A012A012A012A012A012A012A08
:1000A000EC29EC29EC29EC29EC29EC29EC29EC29A8
:1000B000EC29EC29012A012A012A012A012A012A14
:1000C000012A012A1A292329E728012A4F29172959
:1000D0001D29012A012A012A52292029012A012A3F
:1000E0002629012A1429CD28012A012A012A012AB8
:1000F000E128012A012A012A012A012A012A012ACA
:10010000012A012A012AD928012A012ADD28012AE7
:10011000B728012A012A012AEE28012A012A012AE8
:10012000D728012A012AC928CF28012ACB28012A49
:10013000E428012A012A012A012A012A012A012A86
:1001400000302B020319012A24080F398207012AE3
:1001500055295A295F29642969296F2973297E291C
:100160009229A729BC29D129E229E629012AF401EB
:10017000F3018A1500208A01F50000307502031989
:10018000C72875082F23F30A0319F40AB9288A012E
:10019000002A0D24002A3723002A4125002A43087B
:1001A00067233A302F23420867233223002A8D2306
:1001B000002A440867233223002A45086723322394
:1001C000002A35144125002A35104125002A351012
:1001D000E230C5004130C4004125002A28086723C9
:1001E00020302F231F1BF9286F302F236E302F2331
:1001F000FF286F302F2366302F2366302F232808E7
:10020000CB002030A800A80303190B292F261F1BA1
:1002100003292808C9004B08A8002F2620302F23C7
:10022000490867233223002A0130A400FD29023047
:10023000A400FD290330A400FD290430A400FD29F9
:100240000530A400FD290630A400FD2954302F23D9
:1002500069302F236D302F2365302F2372302F23E9
:1002600028302F2330302F232D302F2334302F23CD
:1002700029302F233F302F2332230730A400FD29BC
:100280000830A400FD290930A400FD290A30A4008B
:10029000FD290B30A400FD290C30A400FD290D30F0
:1002A000A400FD290E30A400FD29361AA72925082F
:1002B000A000FD29361ABC292508A100FD29361AFF
:1002C000D1292508A200FD29361A7E292508C30058
:1002D000FD29361A92292508C200C101FD292508E9
:1002E000C4004125FD292508C600361648302F23B5
:1002F0003F302F2332230430A400FD294608C800D4
:10030000C807C807C807C8075030840048088407D2
:10031000250880004D302F233F302F233223053016
:10032000A400FD2925084608C800C807C807C80753
:10033000C8075130840048088407250880005230DF
:100340002F233F302F2332230130A400FD2925081D
:100350004608C800C807C807C807C8075230840045
:10036000480884072508800047302F233F302F237B
:1003700032230230A400FD2925084608C800C8071A
:10038000C807C807C80753308400480884072508F1
:10039000800042302F233F302F2332230330A4002C
:1003A000FD2925084608C800C807C807C807C807A8
:1003B0005430840048088407250880008D233612B5
:1003C0004125FD292508C5004125FD2925081F399E
:1003D000A8002F264125FD2930301A02A300250848
:1003E000A507A507A507A507A507A507A507A507AD
:1003F000A5072308A507AB0A012AA501AB01012A1D
:10040000A40186111F080B110B108B108C130C13F9
:100410000C108C108C127108840070088A002A0E4F
:100420008300A90E290E090083120313850186019A
:1004300083160313051485140515851505128516F5
:1004400005138513831603130614861406118611EB
:1004500006168612061786178316031301308100CD
:100460008113831603139F171F139F129F151F11CC
:100470009F101F10831203139F121F129F151F112D
:100480009F141F10831203130A30A700A703031D34
:10049000462A831203139F08831203130C13831637
:1004A00003139801981798161815831603130C3028
:1004B0009900831603138C018C1683120313980181
:1004C0009817181683120313A401A501AB01A60106
:1004D000B501B601831203138B010B178B17C725C8
:1004E000640083120313810183160313003081001B
:1004F00083120313BF0A45083F02031D9A2A3518C9
:10050000932ABF01C00A44084002031D9A2AC00171
:10051000C10A3C304102031D9A2AC101C20A3C3083
:100520004202031D9A2AC201C30A18304302031D66
:100530009A2AC30150084302031DA92A5108420206
:10054000031DA92A5208A0005308A1005408A200C4
:10055000E42A55084302031DB82A56084202031D27
:10056000B82A5708A0005808A1005908A200E42A98
:100570005A084302031DC72A5B084202031DC72A0B
:100580005C08A0005D08A1005E08A200E42A5F08E4
:100590004302031DD62A60084202031DD62A6108C1
:1005A000A0006208A1006308A200E42A64084302D4
:1005B000031DE42A65084202031DE42A6608A00020
:1005C0006708A1006808A200000000000000000009
:1005D000000000001F1F062B861205138513000064
:1005E000000000000000000000000000000000000B
:1005F00000000000000000000000000000000000FB
:1006000000000000000000000000212B0310200863
:10061000B00703180D2B86120F2B8616000003104F
:100620002108B1070318162B0513182B0517000016
:1006300003102208B20703181F2B8513212B8517DF
:1006400000007A2A83160313FF30B700B70B292B5B
:100650002B2B981C262B831203130800303E990085
:10066000222308000D302F230A302F23080050309A
:100670002F2361302F236E302F2374302F236530CA
:100680002F236C302F2374302F236A302F236530B3
:100690002F2320302F2363302F236F302F236C30F4
:1006A0002F235F302F2370302F2369302F236330A7
:1006B0002F232D302F2330302F232E302F23373070
:1006C0002F232E302F2334302F23322308002615DA
:1006D000AC00AF016430AC02031C702BAF0A6A2B74
:1006E00000302F020319772B26112F082E23643098
:1006F000AC07AF010A30AC02031C802BAF0A7A2B87
:1007000000302F02031D862B2619882B2F082E233D
:100710000A30AC072C082E23080030302F2320305D
:100720002F23500867233A302F23510867232030A6
:100730002F235208672320302F23530867232030AC
:100740002F235408672320302F2320302F233130CC
:100750002F2320302F23550867233A302F235608A4
:10076000672320302F235708672320302F23580872
:10077000672320302F235908672320302F23203070
:100780002F2332302F2320302F235A0867233A306B
:100790002F235B08672320302F235C08672320303A
:1007A0002F235D08672320302F235E086723203026
:1007B0002F2320302F2333302F2320302F235F0887
:1007C00067233A302F236008672320302F236108E6
:1007D000672320302F236208672320302F236308EC
:1007E000672320302F2320302F2334302F23203035
:1007F0002F23640867233A302F23650867232030AE
:100800002F236608672320302F23670867232030B3
:100810002F236808672332230800831203137230E2
:100820002F2365302F2364302F233D302F232008C2
:10083000672320302F2367302F2372302F2365301A
:100840002F2365302F236E302F233D302F23210897
:10085000672320302F2362302F236C302F237530F5
:100860002F2365302F233D302F2322086723322387
:10087000831203130800831203130A30CE00CE0B39
:10088000532C20302F2346302F2346302F23613026
:100890002F2369302F236C302F2365302F236430B2
:1008A0002F23322308003308831603139B0083127F
:1008B00003133408831603139A001C1555309D004A
:1008C000AA309D009C1483120313FF30CD008312C5
:1008D0000313000000000000000000000000000002
:1008E0000000000000000000000000000000000008
:1008F0000000CD0BAB2C8312031377302F23723003
:100900002F2369302F2374302F2365302F2320307D
:100910002F2374302F2369302F236D302F236F3016
:100920002F2375302F2374302F2320302F23613055
:100930002F2364302F2364302F2372302F23653010
:100940002F2373302F2373302F233D302F23330871
:1009500067233223222D831603139C18672C1C1146
:100960001C141A0883120313CA0034084A0203191C
:1009700008008312031365302F2365302F23703056
:100980002F2372302F236F302F236D302F232030F1
:100990002F2377302F2372302F2369302F23743089
:1009A0002F2365302F2320302F2372302F236530E3
:1009B0002F2373302F2375302F236C302F23743067
:1009C0002F2320302F2361302F2364302F236430D6
:1009D0002F2372302F2365302F2373302F23733052
:1009E0002F233D302F233308672320302F237730E8
:1009F0002F2372302F2369302F2374302F2374302C
:100A00002F2365302F236E302F233D302F233408C2
:100A1000672320302F2372302F2365302F2361303E
:100A20002F2364302F2320302F2362302F23613077
:100A30002F2363302F236B302F233D302F234A0881
:100A400067233223831603131C118312031372309E
:100A50002F2365302F2374302F2372302F237930CA
:100A60002F2332233F2C8312031308008312031316
:100A70003308831603139B001C141A0883120313F4
:100A80000800831203130030B3002008B4003B2495
:100A9000B30A2108B4003B24B30A2208B4003B2463
:100AA000B30A4508B4003B24B30A4408B4003B240D
:100AB000B30A5008B4003B24B30A5108B4003B24E5
:100AC000B30A5208B4003B24B30A5308B4003B24D1
:100AD000B30A5408B4003B24B30A5508B4003B24BD
:100AE000B30A5608B4003B24B30A5708B4003B24A9
:100AF000B30A5808B4003B24B30A5908B4003B2495
:100B0000B30A5A08B4003B24B30A5B08B4003B2480
:100B1000B30A5C08B4003B24B30A5D08B4003B246C
:100B2000B30A5E08B4003B24B30A5F08B4003B2458
:100B3000B30A6008B4003B24B30A6108B4003B2444
:100B4000B30A6208B4003B24B30A6308B4003B2430
:100B5000B30A6408B4003B24B30A6508B4003B241C
:100B6000B30A6608B4003B24B30A6708B4003B2408
:100B7000B30A6808B4003B24B30A3508B4003B2428
:100B8000B30A2808B4003B2483120313080083121D
:100B900003130030B3003625A000B30A3625A100A8
:100BA000B30A3625A200B30A3625C500B30A362596
:100BB000C400B30A3625D000B30A3625D100B30AE3
:100BC0003625D200B30A3625D300B30A3625D40021
:100BD000B30A3625D500B30A3625D600B30A362522
:100BE000D700B30A3625D800B30A3625D900B30A90
:100BF0003625DA00B30A3625DB00B30A3625DC00D9
:100C0000B30A3625DD00B30A3625DE00B30A3625E1
:100C1000DF00B30A3625E000B30A3625E100B30A47
:100C20003625E200B30A3625E300B30A3625E40090
:100C3000B30A3625E500B30A3625E600B30A3625A1
:100C4000E700B30A3625E800B30A3625B500B30A33
:100C500036251F39A8002F26831203130800831698
:100C600003139F169F111F119F101F108312031350
:100C7000281E3D2E831603139F1283120313A81DF3
:100C8000442E831603139F1583120313281D4B2E26
:100C9000831603131F1583120313A81C522E8316E9
:100CA00003139F1483120313281C592E8316031356
:080CB0001F1483120313080056
:10100000083074078A000830730703188A0A8200C0
:101010000D340A34483465346C34703420346D3403
:1010200065346E3475340D340A3442346E346E34A3
:101030006E3445344E345434453452342034733491
:1010400065347434203462346C347534653420343F
:101050004C34453444342034283430342D34323444
:101060003534353429342E340D340A3443346E3457
:101070006E346E3445344E34543445345234203456
:10108000733465347434203463346C346F346334B3
:101090006B342034733470346534653464342034F4
:1010A000283430342D3432343534353429342C342A
:1010B0002034643465346634613475346C3474348B
:1010C00020347E34383430342E340D340A346334D2
:1010D00020347034723469346E34743420346334A0
:1010E0006C346F3463346B3420347334703465344F
:1010F000653464342E340D340A344434203473346B
:1011000065347434203463346C346F3463346B343A
:101110002034743469346D3465347234203464346A
:1011200065346634613475346C347434203473340B
:1011300070346534653464342C34203446343D34A2
:101140003234323436342C34203443343D34363463
:1011500035340D340A3446346E346E346E344534CE
:101160004E3454344534523420347334653474343A
:10117000203463346C346F3463346B342034703413
:10118000723465347334633461346C34653472346E
:101190002034283430342D34323435343534293445
:1011A0002C342034643465346634613475346C34E2
:1011B000743420343234353435342E340D340A341A
:1011C000663420347034723469346E3474342034AC
:1011D00063346C346F3463346B3420347034723461
:1011E00065347334633461346C34653472342E3452
:1011F0000D340A3447346E346E346E3445344E3414
:1012000054344534523420347334653474342034C7
:1012100067347234653465346E3420344C3445346C
:1012200044342034283430342D3432343534353499
:1012300029342E340D340A3448346E346E34453437
:101240004E34543445345234203473346534743459
:10125000203468346F347534723420342834303498
:101260002D343234333429342E340D340A344C3492
:10127000203473346534743420346C346934673406
:10128000683474342034733465346E3473346934A0
:1012900074346934763469347434793420342834BD
:1012A00030342D343334313429342C342034643404
:1012B00065346634613475346C34743420343034BD
:1012C0002C342034733461347634653464342034FF
:1012D00069346E342034203445344534503452342B
:1012E0004F344D342E340D340A346C342034703481
:1012F000723469346E34743420346C346934673435
:10130000683474342034733465346E34733469341F
:101310007434693476346934743479342E34203436
:101320006F346E3420346F34723420346F3466344A
:1013300066342034733474346134743475347334E3
:101340002C34203461346E3464342034613463349A
:101350007434753461346C3420346C3469346734DB
:101360006834743420346D346534613473347534C6
:101370007234653464342034283430342D343334BA
:101380003134293420347734683465347234653428
:10139000203430342034693473342034623472346D
:1013A0006934673474346834653473347434203485
:1013B00061346E346434203433343134203469344D
:1013C000733420346434613472346B342E340D340D
:1013D0000A344D346E346E3445344E34543445340E
:1013E0005234203473346534743420346D346934A9
:1013F0006E347534743465342034283430342D34EC
:101400003534393429342E340D340A3450346E34A2
:10141000203445344E3454344534523420347334FB
:10142000653474342034743469346D346534723402
:1014300020346E3475346D34623465347234203443
:10144000283430342D34343429342C342034753459
:1014500073346534203432343534353420346634D2
:101460006F347234203468346F34753472347334AA
:1014700020346F34723420346D3469346E347534F2
:10148000743465347334203474346F3420346434E9
:1014900069347334613462346C34653420346134BB
:1014A0002034743469346D34653472342E340D3420
:1014B0000A3470342034733468346F347734203411
:1014C000743469346D346534723473342E340D34AD
:1014D0000A3452346E346E346E3445344E345434DF
:1014E00045345234203473346534743420347234C7
:1014F0006534643420344C34453444342034283446
:1015000030342D3432343534353429342E340D34DE
:101510000A345334203473346134763465342034DF
:10152000733465347434743469346E3467347334AA
:10153000203469346E3420344534453450345234C8
:101540004F344D342E340D340A3473342034703417
:10155000723469346E347434203452344734423433
:101560002E340D340A3474342034703472346934B7
:101570006E3474342034743469346D3465342E34EC
:101580000D340A34763420347034723469346E3455
:1015900074342034763465347234733469346F347F
:1015A0006E342E340D340A34583420347334653498
:1015B00074342034663461347334743420346D34BC
:1015C0006F34643465342C3420346F346E346C34AE
:1015D000793420346C346F346F346B34203461349C
:1015E0007434203468346F347534723473342C346A
:1015F00020346D3469346E34753474346534733426
:1016000020346D347534733474342034623465346A
:1016100020347A34653472346F342C3420342734D7
:1016200046342734203461346E3464342034273413
:101630006634273420347334743469346C346C3435
:10164000203477346F3472346B342034283473345C
:101650006134763465346434203469346E34203433
:1016600045344534503452344F344D3429342E34BB
:101670000D340A34783420346C3465346134763473
:1016800065342034663461347334743420346D34FA
:0E1690006F34643465342E340D340A34003463
:02400E00183F59
:00000001FF
